:100000000C940C060C9429060C9429060C94392E99
:100010000C9429060C9429060C9429060C942906A4
:100020000C9429060C9429060C9466190C94221938
:100030000C9455260C9429060C9429060C94290638
:100040000C9429060C9429060C9429060C94290674
:100050000C9429060C943F1A0C9429060C9429063A
:100060000C9429060C9429060C9429060C94290654
:100070000C9429060C9429060C9429060C94290644
:100080000C9429060C9429060C9429060C94290634
:100090000C9429060C9429060C9429060C94290624
:1000A0000C9429060C9429060C9429060501098054
:1000B000A101850319012AB700150126B700950192
:1000C00075108100C0050C0901A101850419012AE0
:1000D000A002150126A002950175108100C005013E
:1000E0000906A1018506050719E029E71500250184
:1000F0009508750181020507190029EF15002501F2
:1001000095F075018102050819012905950575010C
:100110009102950175039101C00660FF0961A1017B
:100120000962150026FF00952075088102096315F4
:100130000026FF00952075089102C005010906A15F
:1001400001050719E029E7150025019508750181CA
:10015000029501750881010507190029FF15002680
:10016000FF00950675088100050819012905950508
:1001700075019102950175039101C0000000000016
:10018000000000000000000000000000000000006F
:100190000000000000000000000000000000007EE1
:1001A0000F00D4FFFFFFC700000078000000000030
:1001B0000000002A2B2800000000000000000000C2
:1001C00000000000000029000000002C1E34202147
:1001D0002224342627252E362D3738271E1F20218E
:1001E00022232425263333362E37381F04050607ED
:1001F00008090A0B0C0D0E0F101112131415161707
:1002000018191A1B1C1D2F3130232D350405060724
:1002100008090A0B0C0D0E0F1011121314151617E6
:1002200018191A1B1C1D2F3130354C00DA0281FFC2
:10023000D9F1DB20A4A62EAF00A0C000A1C800AE5B
:10024000D580A81FD300408D1420007F3F1F64324B
:1002500014643214783C1E1E140A0541646A7573D6
:1002600074005261697365004C6F77657200446574
:100270006661756C74004C617965723A200080810A
:1002800082838485868788898A8B8C8D8E8F9091D6
:10029000929394A0A1A2A3A4A5A6A7A8A9AAABAC37
:1002A000ADAEAFB0B1B2B3B4C0C1C2C3C4C5C6C7AE
:1002B000C8C9CACBCCCDCECFD0D1D2D3D4000001C7
:1002C0000101010101010101020202020202020216
:1002D00002030303030303030304040404040404E8
:1002E00005050505050606060606070707070708AC
:1002F000080808090909090A0A0A0B0B0B0C0C0C5F
:100300000D0D0D0E0E0E0F0F0F10101111111212F8
:1003100013131414151516161717181819191A1A75
:100320001B1B1C1D1D1E1E1F2020212222232424D6
:10033000252626272829292A2B2C2D2D2E2F303112
:100340003232333435363738393A3B3C3D3E3F4024
:100350004142434445464748494A4C4D4E4F50510F
:100360005354555658595A5B5D5E5F6162646566C9
:1003700068696B6C6D6F7072737577787A7B7D7E50
:100380008082838587888A8C8E8F91939596989AA0
:100390009C9EA0A2A3A5A7A9ABADAFB1B3B5B7BAB8
:1003A000BCBEC0C2C4C6C9CBCDCFD1D4D6D8DBDD8C
:1003B000DFE2E4E7E9EBEEF0F3F5F8FAFDFFFFAA80
:1003C0007F55402223252628292A2C2D2F303233F1
:1003D0003536383A3B3D3E4042434547494A4C4E0C
:1003E0005051535557595A5C5E6062646668696B38
:1003F0006D6F71737577797B7D7F81838587898A3E
:100400008C8E90929496989A9C9E9FA1A3A5A7A843
:10041000AAACAEAFB1B3B4B6B8B9BBBCBEBFC1C273
:10042000C3C5C6C7C9CACBCCCDCED0D1D2D2D3D406
:10043000D5D6D7D7D8D9D9DADADBDBDBDCDCDCDC24
:10044000DCDDDDDDDDDCDCDCDCDCDBDBDBDADAD9F2
:10045000D9D8D7D7D6D5D4D3D2D2D1D0CECDCCCB74
:10046000CAC9C7C6C5C3C2C1BFBEBCBBB9B8B6B492
:10047000B3B1AFAEACAAA8A7A5A3A19F9E9C9A9822
:10048000969492908E8C8A89878583817F7D7B79F3
:10049000777573716F6D6B6968666462605E5C5AD4
:1004A0005957555351504E4C4A4947454342403E97
:1004B0003D3B3A3836353332302F2D2C2A29282629
:1004C00025232200AF00AE2B0014001A00080015EF
:1004D000001700E00004001600070009000A00E110
:1004E000001D001B000600190005000000000000B0
:1004F00000E300105F2C002A00130012000C00180B
:10050000001C00340033000F000E000D000B00290A
:100510000038003700360010001100000000000015
:1005200000E600115F28002B001E001F00200021A4
:10053000002200E00000000000000000000000E1D8
:1005400000000000000000000000000000000000AB
:1005500000E30001002C002A0027002600250024CB
:10056000002300000000004F005200510050000026
:10057000000000000000000000000000000000007B
:1005800000E600010028002B001E021F02200221AD
:10059000022202E00000000000000000000000E174
:1005A000000000000000000000000000000000004B
:1005B00000E30001002C002A002702260225022465
:1005C0000223023500310030002F002E002D0035AF
:1005D00002310230022F022E022D02000000000024
:1005E00000E60001002800005C00000000000000A0
:1005F000000000C25CC55CC75CC95C00000000C3B1
:100600005CC65CC85CCA5C00000000000000000022
:1006100000E30001002C00000000000000000000CA
:1006200000000000000000000000000000000000CA
:1006300000000000000000000000000000000000BA
:1006400000E6000100280009025B00030100A0FA97
:100650000904000001030101000921110100012228
:10066000400007058103080001090401000203009E
:100670000000092111010001222200070582032048
:100680000001070503032000010904020001030023
:100690000000092111010001226D000705840320DB
:1006A0000001120100020000000853460100010091
:1006B000010200010C0343006F0072006E00650030
:1006C0000000100366006F006F007300740061008B
:1006D0006E000000040309040000000000003E5BFF
:1006E0004F5B3E003E6B4F6B3E001C3E7C3E1C0051
:1006F000183C7E3C18001C577D571C001C5E7F5E1A
:100700001C0000183C180000FFE7C3E7FF000018BA
:1007100024180000FFE7DBE7FF0030483A060E0030
:10072000262979292600407F05050700407F0525F9
:100730003F005A3CE73C5A007F3E1C1C0800081C46
:100740001C3E7F0014227F2214005F5F005F5F0069
:1007500006097F017F00006689956A00606060601D
:10076000600094A2FFA2940008047E0408001020F8
:100770007E20100008082A1C0800081C2A0808000F
:100780001E10101010000C1E0C1E0C0030383E38CD
:100790003000060E3E0E06000000000000000000C3
:1007A0005F000000000700070000147F147F1400A2
:1007B000242A7F2A12002313086462003649562037
:1007C0005000000807030000001C22410000004107
:1007D000221C00002A1C7F1C2A0008083E08080072
:1007E0000080703000000808080808000000606001
:1007F00000002010080402003E5149453E0000421E
:100800007F4000007249494946002141494D33006B
:100810001814127F10002745454539003C4A4949C4
:10082000310041211109070036494949360046493E
:1008300049291E00000014000000004034000000A0
:10084000000814224100141414141400004122144E
:1008500008000201590906003E415D594E007C1214
:1008600011127C007F49494936003E414141220036
:100870007F4141413E007F49494941007F090909C3
:1008800001003E41415173007F0808087F0000418C
:100890007F4100002040413F01007F0814224100B9
:1008A0007F40404040007F021C027F007F04081010
:1008B0007F003E4141413E007F09090906003E415B
:1008C00051215E007F091929460026494949320015
:1008D00003017F0103003F4040403F001F204020B4
:1008E0001F003F4038403F006314081463000304B6
:1008F000780403006159494D4300007F41414100A4
:10090000020408102000004141417F00040201025E
:10091000040040404040400000030708000020540D
:10092000547840007F284444380038444444280028
:10093000384444287F0038545454180000087E0975
:1009400002001824241C78007F0804047800004466
:100950007D4000002040403D00007F102844000002
:1009600000417F4000007C04780478007C08040487
:1009700078003844444438007C1824241800182493
:1009800024187C007C0804040800485454542400B3
:1009900004043F4424003C4040207C001C204020B4
:1009A0001C003C4030403C004428102844004C903F
:1009B00090907C004464544C440000083641000090
:1009C0000000770000000041360800000201020428
:1009D00002003C2623263C0000000000000000002E
:1009E0000000000000000000C0E0F0F8F81800C0AF
:1009F000F0FCFEFFFFFFFFFFFFFF7E000000000096
:100A00000000000080C0E0E0E0E0E0E0E0E0C08066
:100A10000000000080C0E0E0E0E0E0E0E0E0C08056
:100A2000000000E0E0C0C0E0E0E0E00000E0E0C086
:100A3000C0E0E0E0E0E0C0800000000080C0E0E056
:100A4000E0E0E0E0E0E0C080000000000000000026
:100A5000000000000000E0F0F0F0E0ECEEF7F370D2
:100A600020007C7C7C7E007E7E7E7F7F7F000080FD
:100A7000C0E07E5B4F5BFEC00000C000DCD7DEDE66
:100A8000DED7DC00C0000000000000000000000015
:100A90000000000000000000000000000000000056
:100AA00000F8FCFEFFE000FFFFFFFFFFFF80FFFFFD
:100AB000FFFFFFFFFFFFFF1F070100000000000016
:100AC000000000FFFFFF8100000000000081C3C3A1
:100AD000C30000FFFFFF8100000000000081FFFF56
:100AE000FF0000FFFFFF01000000000000FFFFFF0C
:100AF000010000000001FFFFFF0000FFFFFF9D1C41
:100B00001C1C1C1C1C9DDFDFDF000000000000001F
:100B10000000000000000F1F3F7F7F7F7F7F3F1E90
:100B20000C001F1F1F3F003F3F3F7F7F7F00307B38
:100B30007F7830202030787F3B0003000F7F0F0F3D
:100B40000F7F0F0003000000000000000000000005
:100B50000000000000000000000000000000000095
:100B600000030F1F3F3F3F3F1F1F3F3F7F7F7F3FE0
:100B70003F1F3F7F7F7F7F7C7878381C0F0000000D
:100B80000000000001030707070707070707030125
:100B90000000000001030707070707070707030115
:100BA000000000070707000000000000000707071B
:100BB000000000000000070707000000010307070E
:100BC00007070707070703010000000000000000F7
:100BD0000000000000000000000000000000000015
:100BE0000000000000000000000000000000000005
:100BF00000000000000000000000000000000000F5
:100C000000000000000000000000000000000000E4
:100C1000000000000000000011241FBECFEFDAE04A
:100C2000DEBFCDBF12E0A0E0B1E0E6EFF6E602C025
:100C300005900D92AC30B107D9F726E0ACE0B2E0F8
:100C400001C01D92A333B207E1F70E947C260C94E9
:100C500041330C940000FC01AC014C5F5F4F8FEFFF
:100C600091E32191822728E030E087FF09C0880FB7
:100C7000892721503109C9F7E417F50791F708953D
:100C8000880FF7CFE8EDF0E080818E7F80831092AF
:100C9000E2001092DA001092E100A0EEB0E08C9138
:100CA00081608C9380818F77808319BCA7EDB0E041
:100CB0008C918E7F8C9380818F7E80831092F50340
:100CC00008952091E4003091E50095E6A901209176
:100CD000EC00822F817020FF06C08091E80080FF29
:100CE00006C080E008952091E80022FD1AC080919E
:100CF0001A04882389F0853089F08091EB0085FD06
:100D00000FC02091E4003091E50042175307F9F23B
:100D10009150E1F684E0089582E0089583E008951B
:100D200081E00895EF92FF920F931F93CF937C0180
:100D30008B010E946106C82F811117C08091E800C5
:100D400085FD0BC08091E8008E778093E8000E94BB
:100D50006106882399F3C82F08C0F70181917F01AC
:100D60008093F1000150110949F78C2FCF911F9109
:100D70000F91FF90EF90089580911C0487FF13C09E
:100D80008091E80082FF06C08091E8008B77809315
:100D9000E80004C080911A048111F2CF0895809177
:100DA0001A048823D9F38091E80080FFF8CF80915E
:100DB000E8008E77ECCF982F9093E900242F762FC0
:100DC00050E0891731F07091EC002091ED005091C6
:100DD000F00021FD07C09F5F973071F78093E90015
:100DE00081E008953091EB003E7F3093EB0030912D
:100DF000ED003D7F3093ED003091EB00316030939A
:100E0000EB007093EC002093ED005093F0002091E4
:100E1000EE0027FDE0CF80E00895B0E0A0E0E3E140
:100E2000F7E00C94732FC8EDD0E088818F7E888323
:100E3000E7EDF0E080818160808384E082BF81E023
:100E40008093F50388818E7F888302EE10E0F8019D
:100E500010821092DA0081EEC82ED12CF601108299
:100E600088818F77888388818068888388818F7D57
:100E7000888319BC10921A0410921B041092190452
:100E80001092180490EEE92EF12CF70180818B7FEF
:100E9000808388818160888342E060E080E00E94F6
:100EA000DB06F60180818E7F8083F801808181607E
:100EB0008083808188608083F70180818E7F80833A
:100EC000888180618883CDB7DEB7E8E00C948F2FEE
:100ED000FC01809122049091230486179707A0F0CB
:100EE0006115710529F49091E8009E779093E800D0
:100EF00090E06115710551F4911108C08091E800EE
:100F000082FF34C080E00895BC01F2CF80911A04C2
:100F10008823C1F18530C1F18091E80083FD30C0A4
:100F20008091E80082FDEACF8091E80080FFE1CF68
:100F30008091F3002091F200382F6115710519F0AE
:100F40002830310558F091E02830310509F090E063
:100F50002091E8002E772093E800CBCF81918093F9
:100F6000F100615071092F5F3F4FE7CF80911A0464
:100F7000882341F0853041F08091E80083FFBECFA7
:100F800081E0089582E0089583E00895089508952A
:100F900008958091F703089587E797E790930108F4
:100FA0008093000888E19AE00FB6F894A8958093A2
:100FB00060000FBE90936000FFCF2FB7F894609150
:100FC000EC037091ED038091EE039091EF032FBF3E
:100FD0000895209147012223C9F02091F00327FFB3
:100FE00015C0E62FE695E695E695EE31D8F4E80FC4
:100FF000F92FF11D677021E030E001C0220F6A95E2
:10100000EAF720958281282322830895FC013296F5
:1010100008962191621303C0DF0111971C92E81713
:10102000F907B9F70895209147012223C1F02091D3
:10103000F00327FF14C0E62FE695E695E695EE311E
:10104000F8F4E80FF92FF11D677021E030E001C0DE
:10105000220F6A95EAF78281822B82830895FC0130
:1010600032962FEF30E04191641751F02F3F19F481
:10107000411101C0232F3F5F3630A9F72F3F09F4FC
:101080000895820F911D27FD9A95FC0162830895B2
:101090002091E9033091EA032817390771F0909302
:1010A000EA038093E903E091E703F091E8033097C6
:1010B00021F00084F185E02D099508952091E50344
:1010C0003091E6032817390771F09093E603809377
:1010D000E503E091E703F091E803309721F0068003
:1010E000F781E02D09950895FA01811101C0FB01F6
:1010F00009950895E3E3F3E011828281846082839D
:1011000008958091DA03982F9E7F61F48170826048
:101110008093DA038091DD03893718F088E78093A4
:10112000DD0308958634B0F381708464F1CFAF920B
:10113000BF92DF92EF92FF920F931F93CF93DF93B3
:10114000082F162FE901E42FF0E0E254FD4F611162
:1011500010C0E4915E2F4E2F4983E8835A83DF91BC
:10116000CF911F910F91FF90EF90DF90BF90AF90C4
:101170000895E62EF12C4491D42EE42FF0E026E0E1
:10118000829FC00111242FEF30E0B9010E94552F3A
:10119000802F90E0880F991F55E5569FD001579FEB
:1011A000B00D11248A1B9B0B982F990F890F5901A1
:1011B000AE18BF08AE9ED001AF9EB00DBE9EB00D62
:1011C00011245B2F189F80011124012F1127590131
:1011D000A01AB10AAE9E8001AF9E100DBE9E100DEA
:1011E00011245901A81AB108AE9CC001AF9C900D02
:1011F000BE9C900D1124892F9927281B390B2E9FF7
:10120000C0012F9F900D3E9F900D1124E92F623059
:101210007105A1F050F46115710509F49DCF61309D
:10122000710581F0EB2F512F97CF6430710569F074
:1012300080F06630710509F48FCFF4CFE42F4B2F87
:10124000592F8ACFE42F412F87CFEB2F542F492FCF
:1012500083CF4B2F5D2DE12F7FCF80E00895F89451
:10126000E82FE295EF70F0E031A1282F2F7081E098
:1012700090E001C0880F2A95EAF7982F9095932364
:1012800091A392A1892B82A3789408959091F00361
:1012900092FF06C0282F28712830F9F4877F8460D8
:1012A00093FF06C0282F28712831F1F4877E8461CE
:1012B0002091F10320FF06C0382F38713830D9F45F
:1012C000877F816021FF06C0282F28712831D1F443
:1012D000877E816194FD877E0895282F24712430B4
:1012E000F9F68B7F8860DCCF282F2471243101F739
:1012F0008B7E8861DDCF382F3171313019F78E7FC9
:101300008860E0CF282F2171213121F78E7E8861FE
:10131000E1CFCF93DF93EC0182389105B1F108F072
:1013200040C08133910509F49DC048F5893291058B
:1013300009F48DC08A9709F49CC0C11522E5D20733
:1013400008F0BDC0C11531E5D30708F024C1C83E7F
:10135000D10508F0A3C0C13ED10588F5C83AD10532
:1013600008F08EC0C53AD10508F0F6C0C130D105ED
:1013700031F1209721F1C430D10508F545C08533FE
:10138000910509F45FC0C997C1F68091F00383709D
:1013900009F036C18091F10383FF11C0C9E2D0E0AA
:1013A0000EC0833E910599F170F4803E910501F1E4
:1013B000823E910511F68091F00382FD21C0CE019D
:1013C000DF91CF910895863E910561F1873E9105A9
:1013D00071F1843E910509F0B0CF8091F10381FF56
:1013E000EECF8091F003C7EED0E084FD0DC0E7CFD3
:1013F0008091F00380FD33C09091F10390FFDFCF27
:10140000C3EED0E084FFDBCFD0E0C0E0D8CF809146
:10141000F00382FDF2C09091F10390FDF1C084FFD2
:10142000CECFF2CF8091F00383FDDDCFC8CF809186
:10143000F00383FDE8C09091F10391FFF0CFC4EE7B
:10144000D0E0BDCF8091F00385FFB9CFA7CF8091C9
:10145000F00385FDDBC08091F10383FFB0CFC9E3CA
:10146000D0E0ADCF8091F00386FFA9CFCAE2D0E0F3
:10147000A6CF8091F00386FFA2CFC1E3D0E09FCF3B
:10148000CF3BD10508F6C85AD0E0CC0FDD1FC856B7
:10149000DE4F0990D881C02DD46491CFC11540E5AD
:1014A000D40708F064C0C11580E4D80708F05CC018
:1014B000CE019A9581159F4108F481CFA5CFC11522
:1014C00036E5D30718F5C11545E5D40708F07CC00B
:1014D000C11584E5D80708F072C09E012370332738
:1014E0009C2F96959695C115D34508F459C0C1E037
:1014F000D0E002C0CC0FDD1F2A95E2F730E2939FC7
:10150000C0011124C82BD92BDA6859CFC1158AE53F
:10151000D80778F4C11529E5D20708F060C0C115D5
:1015200038E5D30708F470CFDC2FCC27C06FD06A22
:1015300046CFCE0190568115904208F065CF8D2F91
:101540008F710E94460990E0982F882788279F7105
:101550009C012C2BE90141C0C55AD0E0CB56DE4F8F
:10156000C881D0E0D0642BCFDF70D06A28CFCE0105
:101570008370992721E030E002C0220F331F8A9543
:10158000E2F7C695C69580E2C89FE0011124C22B00
:10159000D32BDD6814CFDC2FCC27C16FD06A0FCFDF
:1015A000C1E0D0E002C0CC0FDD1F2A95E2F720E2B7
:1015B000929FC0011124C82BD92BDC6800CFDC2FEF
:1015C000CC27C46FD06AFBCE8C2F0E944609C82F4F
:1015D000D0E0DC2FCC27CC27DF71D062F0CE8C2F6F
:1015E0008F700E94460934E0D695C7953A95E1F789
:1015F000CF709C2FEC01D069E2CEC2EED0E0DFCEFE
:10160000C0EED0E0DCCEC6EED0E0D9CEC5E3D0E06F
:10161000D6CE80919C02811110929C0208958095F3
:1016200090919B02982390939B0208958091780259
:1016300090914702981301C008958F5F8770FACF89
:10164000292F983078F5863068F590E036E0239FB2
:10165000800D911D1124682F677023E09695879562
:101660002A95E1F7FC01EE0FFF1FE80FF91FE15D7E
:10167000FD4F50E040E080E0219130E0062E02C0B6
:10168000369527950A94E2F721703327042E01C07E
:10169000220F0A94EAF7822B4F5F5F4F43305105C8
:1016A00059F7089580E00895292F983098F58630ED
:1016B00088F590E036E0239F800D911D1124282F9E
:1016C000277041E001C0440F2A95EAF723E0969580
:1016D00087952A95E1F7FC01EE0FFF1FE80FF91F30
:1016E000E15DFD4F30E020E070E05191DF011197A6
:1016F000CB01022E02C0969587950A94E2F781707D
:1017000081958527842385278C932F5F3F4F233036
:10171000310559F70895CF93DF93682F81E06A3040
:1017200019F06D3031F480E00E94190CDF91CF91F7
:101730000895809131069091320626E0FC01ABE2DB
:10174000B6E001900D922A95E1F7603E08F458C08A
:1017500026E0FC0111922A95E9F7C0913106D0915B
:10176000320646E050E0BE018BE296E00E94443033
:101770009E012B523440892B41F1C90145E09695D9
:1017800087954A95E1F741E050E0BA0102C0660F43
:10179000771F8A95E2F7CB016091290470912A04A2
:1017A000862B972BB9016B5F7F4FE5E076956795A8
:1017B000EA95E1F702C0440F551F6A95E2F7842BC2
:1017C000952B90932A04809329042A5F3F4F4091E0
:1017D0002804642F70E0C9010E94552F481B463031
:1017E00010F4240F311D211572E0370710F030E09E
:1017F00020E0255D3B4F309332062093310696CF93
:10180000F6E06F9FB00111246852794F46E050E036
:101810000E942E30A2CFCF93DF93EC01FE01849182
:10182000811103C0DF91CF9108950E948B0B219607
:10183000F5CFCF93382FE0913106F0913206EB527D
:10184000F44020912804622F70E0CF010E94552FB0
:10185000281B822F332361F066E00E94A02FC82F3F
:10186000C15010F4CF91089580E20E948B0BF8CF05
:101870009F01280F311D2115324018F080E0F0E063
:10188000E0E08E0F9F2F911D855D9B4F9093320658
:1018900080933106E7CF80919B0290919A02892B29
:1018A00080930E0290919C029923A1F0892B809342
:1018B0000E02809147018823E1F18091F00387FFB8
:1018C00038C08EE1E0E1F2E090E08150A0F59111A6
:1018D0000E94090B40E250E06AE772E08EE092E07D
:1018E0000E944430892B21F180E2EEE0F2E0AAE789
:1018F000B2E001900D928A95E1F7E091E703F09153
:10190000E8033097A9F080914701882359F080912E
:10191000F00387FF07C080910E0280930F0286E0DC
:1019200080930E020280F381E02D8EE092E0099513
:10193000089586E0C7CF2191222339F29F5FC5CF5A
:1019400090E080E00E945E0890E080E00E944808FD
:1019500010929A020E944B0C0895809327040E94D3
:10196000A00C089580912704982F9670963021F44A
:1019700088600E94AD0C0895877FFBCF21E030E0A6
:1019800001C0220F8A95EAF72095809127048223CF
:101990000E94AD0C089590917902809589238093DF
:1019A0007902282F277091F4282F082E000C330B72
:1019B0009217130659F09091F10392FF07C0859595
:1019C000859585950E94BE0C10927902089521E0BC
:1019D00030E001C0220F8A95EAF780912704822B1C
:1019E0000E94AD0C089580939D020E94A00C089562
:1019F00010929B0280914701E0E1F2E0882361F0C0
:101A00008091F00387FF08C08EE1DF011D928A9567
:101A1000E9F70E94A00C089586E0F7CFAAE2B0E0B3
:101A2000E4E1FDE00C94782F8CE194E02091F1004A
:101A3000DC012D93CD01B4E084329B07B9F780918E
:101A40001D04833009F472C0B8F4813009F449C030
:101A5000823009F4B3C08091E80083FF8BC280918B
:101A60001C0490911D049A3008F084C2E92FF0E024
:101A7000ED5BFC4C0C94F02F8A3009F48EC08B3057
:101A800009F471C0893039F780911C04813219F74B
:101A90008091200490912104009711F00297D9F6CB
:101AA0008091E800877F8093E8008091E80082FFC2
:101AB00038C09091F3008091F200029731F4809148
:101AC000F100813011F0863021F48091F100809393
:101AD000F7038091E8008B778093E8000E94BC06B2
:101AE000BACF80911C04813A09F0B5CF8091E8000B
:101AF000877F8093E8008091200490912104892BB6
:101B000061F460E288EF93E070E00E9468078091E2
:101B1000E8008B778093E8009ECF60E090E080E063
:101B2000F3CF80911A048111C0CF95CF80911C040E
:101B3000813A09F090CF8091200490912104892B63
:101B400009F089CF8091E800877F8093E800809139
:101B5000E80080FFFCCF809147018093F1008091E5
:101B6000E8008E77B9CF80911C04813209F073CFE1
:101B70008091200490912104892B09F06CCF8091F1
:101B8000E800877F8093E8000E94BC0680911E04D5
:101B9000809347010E94F80C5ECF80911C04813233
:101BA00009F059CF8091E800877F8093E8000E9478
:101BB000BC0680911F048093F6034DCF80911C04D6
:101BC000813A09F048CF8091E800877F8093E80050
:101BD0008091E80080FFFCCF8091F603BECF803873
:101BE00099F0823809F0C6C1809120048F70873047
:101BF00008F0C0C18093E9008091EB0085FB882745
:101C000080F91092E90006C080911804909119049F
:101C1000911182609091E800977F9093E800809303
:101C2000F1001092F1008091E8008E779FC1882327
:101C300009F48DC1823009F09DC180911E0481118B
:101C400090C1809120048F702FEF280F263008F06C
:101C500091C18093E9002091EB0020FF82C1933075
:101C600031F48091EB0080628093EB007AC1909117
:101C7000EB0090619093EB0021E030E001C0220F77
:101C80008A95EAF72093EA001092EA008091EB002F
:101C90008860EACF81116EC110911E041F77809178
:101CA000E3008078812B8093E3008091E800877FB8
:101CB0008093E8000E94BC068091E80080FFFCCF82
:101CC0008091E30080688093E30082E0111183E05B
:101CD00080931A044FC18058823008F04BC1209184
:101CE0001E0430911F042C3DE3E03E07A1F583E084
:101CF0008A838AE289834FB7F894DE01139620E045
:101D00003EE051E2E32FF0E050935700E49120FFD2
:101D100003C0E295EF703F5FEF708E2F90E0EA30E6
:101D2000C0F0C7968D939D932F5F243159F74FBF15
:101D30008091E800877F8093E8006AE270E0CE013E
:101D400001960E9468078091E8008B778093E800F5
:101D500011C1C096E7CF8091200490912104432FB8
:101D600055274330510509F44AC078F541305105F3
:101D700009F47AC08BE590E0E7E4F6E042305105E3
:101D800009F0F8C02091E800277F2093E800209117
:101D90002204309123048217930708F49C0140E049
:101DA0002115310509F065C0411163C08091E8003B
:101DB00082FDC9CF80911A04882329F2853019F257
:101DC0008091E80083FFF2CFBECF4132510509F484
:101DD0003CC04232510509F0CDC08330910508F076
:101DE000C9C0FC01EE0FFF1FE050FE4F0190F081D3
:101DF000E02D83509E4FDC018C9190E01AC0332778
:101E000021303105D1F02115310561F02230310545
:101E100009F0B0C0E4EBF6E0E4918E2F90E0E4EB43
:101E2000F6E007C0E4EDF6E0E4918E2F90E0E4EDFB
:101E3000F6E0009709F49EC0A5CFE2ECF6E0E4914D
:101E40008E2F90E0E2ECF6E0F4CF8330910508F0BD
:101E500091C0880F991FFC01EA5FFD4F0190F0814E
:101E6000E02D89E090E08ECF82E190E0E2EAF6E0BA
:101E700089CF80911A04882309F465CF853009F44D
:101E800062CF8091E80083FD5ECF8091E80082FD03
:101E90008DCF8091E80080FF83CF9091F3008091F7
:101EA000F2002115310519F08830910550F041E01C
:101EB000089709F040E08091E8008E778093E80071
:101EC0006FCF44914093F100319621503109019632
:101ED000E8CF803809F04EC08091E800877F80937A
:101EE000E80080911B048093F1009DCE811142C0D7
:101EF00010911E041230F0F58091E800877F8093E6
:101F0000E80010931B040E94BC06112311F084E02A
:101F100005C08091E30087FDFACF81E080931A0429
:101F200042E061EC81E00E94DB0642E261EC84E089
:101F30000E94DB0642E261EC82E00E94DB0642E2A4
:101F400060EC83E00E94DB0680911A0413C080914C
:101F50001E04813079F481E0933009F080E08093B1
:101F600019041092E9008091E800877F8093E800CF
:101F70000E94BC068091E80083FF0AC08091E800BF
:101F8000877F8093E8008091EB0080628093EB0074
:101F9000AA96E3E00C94942F882321F00E940F0B63
:101FA0000E944B0C0895882339F090919B02982B46
:101FB00090939B020E944B0C0895882351F19CEF53
:101FC000980F913A40F4682F8EE092E00E94E90762
:101FD0000E944B0C089590E2980F983050F487704F
:101FE00091E001C0990F8A95EAF7892F0E940F0BA3
:101FF000EFCF9BE5980F933028F490E080E00E94AB
:102000005E080895885A873120F490E080E00E94AD
:1020100048080895CF93C82F8823D9F18CEF8C0FEF
:10202000813AC8F580914701882311F18091F0032E
:1020300087FF1EC0EC2FE695E695E695F0E0E25F9F
:10204000FD4F828190E04C2F477021E030E002C0CC
:10205000220F331F4A95E2F782239323892B91F0B5
:102060006C2F8EE092E00E94E9070E944B0C0AC0A0
:10207000E0E1F2E086E192E02191C21789F38E1748
:102080009F07D1F76C2F8EE092E00E9413080E9408
:102090004B0CCF91089580E28C0F883068F4C770A4
:1020A00021E030E001C0220FCA95EAF780919B023F
:1020B000822B80939B02EBCFEBE5EC0FE33040F4F7
:1020C000F0E0EB56FE4F808190E00E945E08E1CF89
:1020D000C85AC731F0F6EC2FF0E0EE0FFF1FE856BC
:1020E000FE4F808191810E944808D3CFB0E0A0E0EC
:1020F000ECE7F0E10C94732F6C017B0164E670E077
:1021000088E70E94B32CEC0197FD12C010E000E0BC
:10211000F601E00FF11F849164E670E00E941F2D2C
:10212000EC01892B29F40F5F1F4F0E151F0581F756
:102130000E94952DCE01CDB7DEB7E8E00C948F2F2D
:102140008091E3039091E403911103C091E089270A
:102150000895882369F062E070E085EC94E00E94C5
:102160007610892B19F08091E30308951092E30310
:102170008091E303EBCFCF93C091E3038091E4031D
:102180008823D1F00E94DD07605A75418F4F9F4F21
:102190006093DF037093E0038093E1039093E20385
:1021A000C11108C062E070E083EC94E00E947610F8
:1021B000892B29F0C091E3038C2FCF91089581E002
:1021C0008093E303F7CF8093F2037093F40360935B
:1021D000F30380911A048430F9F48093E9008FEFBF
:1021E0009091E800815095FD06C095ED9A95F1F724
:1021F00000008111F5CF8091E80085FF0DC050E00F
:1022000040E063E070E082EF93E00E9492068091EC
:10221000E8008E778093E8000895BC0184E00E9476
:10222000E3100895BC0183E00E94E3100895CF936A
:10223000DF93EC01809147018823B1F18091F00395
:1022400087FF32C060E284E08093E9008FEF9091D5
:10225000E800815095FD06C095ED9A95F1F70000D4
:102260008111F5CF8091E80085FF1BC08091470167
:1022700070E050E040E0811104C050E040E068E0D0
:1022800070E0CE010E9492068091E8008E778093E4
:10229000E80080E2FE01A8EFB3E001900D928A957C
:1022A000E1F7DF91CF91089568E081E0CDCF6091B3
:1022B00043018091DA0380FF20C08091420143E016
:1022C000849FC0011124885C9C4F539A2BB1277FB7
:1022D0003BB138605FB7F894FC01649FE00DF11DDD
:1022E0001124BF0168177907D1F45FBF8FE594E02F
:1022F0000197F1F700C0000008958091440190918A
:10230000450123E0829FF0011124E85CFC4F89170E
:10231000A0F61182108212828F5F3396F8CFFC01F3
:102320004191CF01E8E03BB9000000C047FF2BB965
:10233000440F000000C000C000C02BB900C0EA95E7
:1023400091F7D0CFB0E0A0E0E8EAF1E10C946F2F74
:10235000EC014C81042F10E09801D8010E94053057
:102360009B01AC010E941B304B015C01E0E2F0E0FC
:10237000E01BF10BA5E5B0E0AC019B010E941B3016
:102380006B017C019F01DF010E94FD2F9B01AC01CD
:102390000E9426309B01AC01280D391D4A1D5B1D92
:1023A000C701B6010E94CE2FF22E822F90E039E2B3
:1023B0003F1520F143E0249F900111243595279586
:1023C000122F109500E085E5E82EEF188091460168
:1023D000081718F10E9457119C8181E0992319F088
:1023E000903219F48FEF8093410180914101890F60
:1023F0008C83CDB7DEB7ECE00C948B2F25E530E075
:10240000B901681B790B9B01220F331F260F371F61
:1024100037FFD4CF2F5F3F4FD1CF8E2D01FD8F2DB2
:1024200020914401622F600F7727771F9B01220FB5
:10243000331F260F371F285C3C4F412F193708F0F8
:1024400048E76091DC030E9497080F5FBFCFEF92CF
:10245000FF920F931F93CF93DF93EC018C81811137
:1024600009C081E08C831092370392E09093400181
:1024700080933F01809144019091450123E0829F28
:10248000F0011124E85CFC4F891758F110E003E0DB
:1024900060914601161758F10E94571180913F0133
:1024A00020913703280F2093370390914001980F14
:1024B00090934001191654F4022E000C330B4091F6
:1024C00046014150550B2417350734F08195809310
:1024D0003F01813009F41C82CDB7DEB7E6E00C94F1
:1024E000912F1182108212828F5F3396CDCFE12E11
:1024F000F12C70E0C7010E94BA2F20914401820F95
:10250000482F50E020913703022E000C330BE216C7
:10251000F306D4F020914001022E000C330B2E154F
:102520003F0594F0809F90011124285C3C4F40911E
:10253000DD03493708F048E76091DC038091DB0355
:102540000E9497081F5FA4CFFA01EE0FFF1FE40F50
:10255000F51FE85CFC4F118210821282F3CFB0E0CD
:10256000A0E0E5EBF2E10C946F2FEC018A81BB2433
:10257000BA9480FD02C0BB24B394A09046018C8124
:10258000811109C081E0B81220C08FEF8A0D8093BD
:10259000360381E08C83F12CE12C46E3842EEA148F
:1025A000B8F00E9457118091360391E0B9125AC0D9
:1025B000811153C0809146018150809336031C8263
:1025C000CDB7DEB7ECE00C948B2F10923603E1CF41
:1025D000009144010E0D1F2D111DC801880F991F78
:1025E000080F191F085C1C4FF8011182108212821B
:1025F00034E0C32ED12C912C80913603890D873382
:1026000044F1682D0E94AC2F892F082E000C990BE5
:102610008E159F05A9F48091DD038C9DA0018D9DF1
:10262000500D11245595479555954795493708F014
:1026300048E798016091DC038091DB030E949708D2
:102640009B0CF1E0CF1AD108B9F68FEFE81AF80A1F
:10265000A6CF87FFDACF8A0DD8CF8150809336037B
:10266000BC82AECF90E001966091460170E00E947E
:10267000BA2F809336038C83A3CFEF92FF921F93E0
:10268000CF93DF93EC0110E0EE24EA94F12C6091FB
:102690004601161770F00E9457119A818C8190FFA5
:1026A0002AC08F5F8C83DF91CF911F91FF90EF90B5
:1026B000089520914401422F410F5527551FCA010B
:1026C0009A01220F331F280F391F285C3C4F40917D
:1026D000DD03493708F048E770E0C7010E94BA2FD0
:1026E000962F8C816091DC03199F800D11240E942C
:1026F00097081F5FCCCF8150D5CF9091DA0390FF20
:102700000EC0909144012091450133E0939FF00168
:102710001124E85CFC4F921718F00E94571108959D
:102720008183608342839F5F3396F5CFA3E0B0E05F
:10273000ECE9F3E10C94792F9091DA0390FF0DC04E
:10274000493708F048E79E012F5F3F4F0E949708E6
:102750004B8169818A810E947D132396E2E00C946B
:10276000952FCF93DF93EC01EAEDF3E04381628193
:102770008C810E9496138C818F5F8C83DF91CF9127
:102780000895CF93DF93EC01EC81F0E0ED53FC4F23
:102790004491EAEDF3E0628181810E9496138C817D
:1027A0008F5F8C83DF91CF910895EAEDF3E0808114
:1027B0008E7F80830E947A08E3E3F3E08281816068
:1027C00082832FEF80E792E0215080409040E1F734
:1027D00000C000000E9457110895B0E0A0E0E3EFB0
:1027E000F3E10C94712F7C015B016A018091CA02B4
:1027F00001E010E08A3010F40AE010E0C1E0D0E01F
:10280000B501C701F6010995811104C021960C1785
:102810001D072CF4CDB7DEB7EAE00C948D2FCC9FCA
:102820009001CD9F300D300D112490E080E045E304
:102830004A95F1F70000019682179307C1F7E0CFA0
:102840008091A802811119C088EC90E02091E300EA
:1028500027FD10C0EFE3FCE93197F1F700C000005D
:102860000197A1F782E08093A8020E94420610928D
:102870001A0403C081E08093A80281E09091A8022D
:10288000913011F080E0089508950E94201488236B
:1028900059F0E091E703F091E803309729F00190B7
:1028A000F081E02D0995089580E008950F931F931E
:1028B0000E942014882329F00E94DD071F910F91A8
:1028C00008950E94DD070091CB021091CC02209167
:1028D000CD023091CE02600F711F821F931FEECF89
:1028E0001F93CF93DF93182FD0E0C0E0893311F40A
:1028F000C0E5D0E0812F0E940A10209739F4812F83
:102900000E94DD0FDF91CF911F9108958FE99FE025
:102910000197F1F700C000002197EFCF0E94F80C5B
:102920002FEF84E39CE0215080409040E1F700C00D
:10293000000088E19AE00FB6F894A89580936000B3
:102940000FBE90936000FFCFCF93DF93C7EAD1E033
:1029500060E0CE010E940D332196C11584E0D807B6
:10296000B9F7DF91CF9108951F93CF93DF93122F83
:102970008430E0F46830D0F44630C0F4C42FD0E0A6
:10298000CC0FDD1F9CE0699FC00DD11D112490E686
:10299000899FC00DD11D1124632FCE0187960E94FF
:1029A0000D33612FCE0188960E940D33DF91CF91B8
:1029B0001F910895AF92BF92CF92DF92EF92FF9254
:1029C0001F93CF93DF9387ECC82E84E0D82ED0E0FE
:1029D0007601C0E014C0F50125913491412F6C2F90
:1029E0008D2F0E94B41482E0A80EB11C1F5F163018
:1029F00091F78CE0E80EF11CCF5FC83019F0570159
:102A000010E0E9CFDF5F80E6C80ED11CD43001F7BB
:102A1000DF91CF911F91FF90EF90DF90CF90BF900B
:102A2000AF900895CF93C82F6FEF811163E283E2D7
:102A300090E00E940D33C1110DC0CFEF6C2F84E2E6
:102A400090E00E940D336C2F85E290E00E940D33E0
:102A5000CF910895C3E0F2CF80E00E94121560E0AC
:102A600086E290E00E940D330E94DA140E94A414C2
:102A700081E00E9412150895CF93C091F103C2FB2B
:102A8000992790F9981791F080FBC2F9C093F10350
:102A90006091F00384E090E00E940D336C2F82E29D
:102AA00090E00E940D3382E00E94CB0CCF910895FC
:102AB0000F931F93CF93DF93843030F5683020F568
:102AC000463010F5C42FD0E0CC0FDD1F2CE0629F04
:102AD000C00DD11D112430E6839FC00DD11D1124DE
:102AE000CE0187960E94F932082F10E0102F0027A0
:102AF000CE0188960E94F9329801282BC901DF91F6
:102B0000CF911F910F91089590E080E0F8CF462F6C
:102B1000843040F4783030F4663020F4672F0E941F
:102B20005815089590E080E00895CF92DF92FF92CB
:102B30000F931F93CF93DF936C0100912704809133
:102B40009D02082BC7E0D0E010E0FC2EC8010C2E3F
:102B500002C0959587950A94E2F780FD0CC02197F5
:102B6000A0F7F12C8F2DDF91CF911F910F91FF9046
:102B7000DF90CF900895B6018C2F0E9487150E9498
:102B80008909019761F3EECFCF93DF93EC010E94A7
:102B90009515BE010E9487150E948909DF91CF918A
:102BA0000895FC0183819481892B29F08081918192
:102BB00089238F3F51F480E00895843FE1F717C0E7
:102BC000883EA8F0813FB9F712C0808191810E94B0
:102BD000C41592959F70963099F358F4925F9F7048
:102BE000923048F7803F19F040F7883E20F781E0A7
:102BF00008959A5FF4CF83E290E00E94F932833225
:102C000089F484E290E00E94F932833059F485E23D
:102C100090E00E94F93291E0833009F090E0892F32
:102C20008170089580E0FCCFCF9384E090E00E9413
:102C3000F932C82F82E290E00E94F932982F8C2F4F
:102C4000CF910895CF92DF92EF92FF926B017C01BA
:102C50000E948108B701A60188E090E00E941F331E
:102C6000FF90EF90DF90CF900895A3E0B0E0EBE30A
:102C7000F6E10C94722FF82ED62E042FC22E9091CE
:102C8000DA0390FF3EC0E92FE695AE2FB0E0A652E2
:102C9000BE4F8C91809333039E7F9230B1F54937BC
:102CA00008F048E79E012F5F3F4F6D2D8F2D0E944A
:102CB00097084B8169818A810E947D138091DB0393
:102CC0008F1108C08091DC038D1104C08091DD0359
:102CD000801729F080913503826080933503F0924C
:102CE000DB03D092DC030093DD03CC2051F0609134
:102CF000DA037091DB038091DC039091DD030E9485
:102D000022162396E9E00C948E2F823019F400915C
:102D1000DD03D4CF863019F4F090DB03CFCF8930B8
:102D2000D9F3893159F6E9516E2F6170B62EE695C7
:102D3000F0E0E254FC4F1491E12C60914601E6165C
:102D400018F00E945711BACFE19EC001112470E023
:102D50000E94552F8F2DB11017C0860F209144016E
:102D6000622F6E0D7727771F9B01220F331F260FCF
:102D7000371F285C3C4F402F093708F048E76D2D7E
:102D80000E949708E394D9CF861BE8CFEAEDF3E0E1
:102D9000438121E1421B08F440E021E0628181810E
:102DA0000E9435160895EAEDF3E0438121E1420FD8
:102DB00008F44FEF21E0628181810E943516089569
:102DC000EAEDF3E0628121E1621B08F460E021E0BA
:102DD000438181810E9435160895EAEDF3E0628116
:102DE00021E1620F08F46FEF21E0438181810E94AD
:102DF00035160895EAEDF3E0818121E04381628197
:102E00008A500E9435160895EAEDF3E0818121E0B1
:102E100043816281865F0E94351608958091DE03AA
:102E2000882319F081508093DE036091DA0370915A
:102E3000DB038091DC039091DD030E94221608954C
:102E40008091DE03833018F48F5F8093DE036091FE
:102E5000DA037091DB038091DC039091DD030E9423
:102E600022160895EAEDF3E083E0808311828FEF6C
:102E7000828388E783831482A3E3B3E012968C9164
:102E80001297836012968C93608171818281938105
:102E90000E942216089568EE7EEF90E080E00E9486
:102EA0002B3360E082E090E00E940D3360E083E02D
:102EB00090E00E940D3310929D0260E084E090E06B
:102EC0000E940D3364E082E290E00E940D3360E0E6
:102ED00085E090E00E940D3360E086E090E00E9483
:102EE0000D336FEF87E090E00E940D3340E050E03B
:102EF000BA0188E090E00E941F3360E08DE090E02E
:102F00000E940D3340E050E0BA0188E190E00E9459
:102F10001F3360E087E190E00E940D3340E050E015
:102F2000BA018CE190E00E941F3370E060E080E223
:102F300090E00E942B3340E050E0BA0188E190E03D
:102F40000E941F3380E00E9412150E942C1540E061
:102F500050E0BA018FE090E00E941F3340E050E063
:102F6000BA0183E190E00E941F330895A4E0B0E02D
:102F7000ECEBF7E10C94782F4091B1025091B20242
:102F80006091B3027091B4022FB7F8948091EC0372
:102F90009091ED03A091EE03B091EF032FBF841B3E
:102FA000950BA60BB70B11E084369105A105B10571
:102FB00070F10E9456146E5F7F4F8F4F9F4F698351
:102FC0007A838B839C8380911101909112018B54A1
:102FD0009D4F4091100150E04530510510F044E004
:102FE00050E0BE016F5F7F4F0E94513082E090E061
:102FF0000E94DF2E182F882351F00E94DD07609376
:10300000B1027093B2028093B3029093B402812F05
:103010002496E3E00C94942FA8E0B0E0E2E1F8E11C
:103020000C94792F85E0EAEDF3E0DE011196019032
:103030000D928A95E1F78091330390913403A0912A
:1030400035038E839F83A88728854091C6025091BF
:10305000C7026091C8027091C9023FB7F89480918D
:10306000EC039091ED03A091EE03B091EF033FBF0D
:10307000841B950BA60BB70B84369105A105B105F2
:1030800010F4222319F18091190190911A018B54A7
:103090009D4F4091180150E04930510510F048E033
:1030A00050E0BE016F5F7F4F0E94513083E090E09F
:1030B0000E94DF2E882369F00E94DD076093C6021C
:1030C0007093C7028093C8029093C902109235038F
:1030D00081E02896E2E00C94952FEF92FF921F93E7
:1030E000CF93DF9300D000D00F92CDB7DEB77B0136
:1030F00090E080E00E94DF2E182F882309F487C01B
:103100004091030150E04115510511F041E050E0BC
:1031100060910401709105016B547D4FCE010596BD
:103120000E9451304091AD025091AE026091AF02C9
:103130007091B0022FB7F8948091EC039091ED0359
:10314000A091EE03B091EF032FBF841B950BA60B4C
:10315000B70B84369105A105B10540F486EB92E0EA
:103160000E942B069D81891709F451C081E090E0EF
:103170000E94DF2E81111AC010E08091A902909167
:10318000AA02A091AB02B091AC02F70180839183B7
:10319000A283B383812F0F900F900F900F900F9009
:1031A000DF91CF911F91FF90EF90089540910B0117
:1031B00050E04530510510F044E050E060910C01C2
:1031C00070910D016B547D4FCE0101960E945130DC
:1031D00086EB92E00E942B069D818913CDCF0E9441
:1031E000DD076093AD027093AE028093AF029093BF
:1031F000B00289819A81AB81BC818093A9029093AE
:10320000AA02A093AB02B093AC0211E0B6CF8091BA
:10321000B6029091B702A091B802B091B902898329
:103220009A83AB83BC831111E4CFA7CF90E080E0F9
:103230000E940733883E9E4F19F40E94FB150895A3
:1032400080E008951F920F920FB60F9211242F93D2
:103250003F934F935F936F937F938F939F93AF931E
:10326000BF93CF93DF93EF93FF93D091E900DF708B
:103270008091EC00C82FC17080FDC0E81092E90079
:103280008091F000877F8093F00078940E940E0D6B
:103290001092E9008091F00088608093F000CD2BBF
:1032A000CF70C093E900FF91EF91DF91CF91BF9173
:1032B000AF919F918F917F916F915F914F913F91CE
:1032C0002F910F900FBE0F901F9018951F920F9285
:1032D0000FB60F9211242F933F934F935F936F93E9
:1032E0007F938F939F93AF93BF93EF93FF938091BF
:1032F000E10082FF09C08091E20082FF05C0809159
:10330000E1008B7F8093E1008091DA0080FF24C090
:103310008091D80080FF20C08091DA008E7F80935A
:10332000DA008091D90080FF9DC080E189BD82E1F3
:1033300089BD09B400FEFDCF81E080931A0480911D
:10334000F503811109C00E9442060E940D07809179
:10335000E20084608093E2008091E10080FF17C06A
:103360008091E20080FF13C08091E2008E7F809305
:10337000E2008091E20080618093E2008091D800B9
:1033800080628093D80019BC85E080931A048091F4
:10339000E10084FF2BC08091E20084FF27C080E120
:1033A00089BD82E189BD89B5982F917080FFFBCFDF
:1033B0008091D8008F7D8093D8008091E1008F7E2E
:1033C0008093E1008091E2008F7E8093E200809103
:1033D000E20081608093E20080911B04882309F45D
:1033E00047C084E080931A0480911A048091E10020
:1033F00083FF27C08091E20083FF23C08091E1001A
:10340000877F8093E10082E080931A0410921B046E
:103410008091E1008E7F8093E1008091E2008E7FB9
:103420008093E2008091E20080618093E20042E0BC
:1034300060E080E00E94DB068091F000886080936D
:10344000F000FF91EF91BF91AF919F918F917F918C
:103450006F915F914F913F912F910F900FBE0F9001
:103460001F90189519BC10921A041092F50374CF8E
:103470008091E30087FD93E090931A04B5CF789490
:103480001F921FB61F9211248F939F93AF93BF93E8
:103490008091EC039091ED03A091EE03B091EF03C6
:1034A0000196A11DB11D8093EC039093ED03A093B1
:1034B000EE03B093EF03BF91AF919F918F911F9057
:1034C0001FBE1F9018959C014FB7F8948091EC0394
:1034D0009091ED03A091EE03B091EF034FBF821BDB
:1034E000930B08952FB7F8948091EC039091ED031E
:1034F000A091EE03B091EF032FBF08950F931F9398
:10350000CF93DF93C62FD42F022FFC018281882313
:10351000A9F0609326040E94721A90932504809368
:103520002404C77081E001C0880FCA95EAF70E94A1
:10353000D30FDF91CF911F910F91089580912604B1
:10354000681332C080912404909125040E94631A6C
:10355000883C910548F510E21D0FCD17B9F080E2C7
:103560008C0F883040F4C77081E001C0880FCA9585
:10357000EAF70E94CC0F183048F481E09D2F977035
:1035800001C0880F9A95EAF70E94D30F802F0E94FE
:103590007014183070F6D77081E001C0880FDA958A
:1035A000EAF70E94CC0FC5CFC77081E001C0880F39
:1035B000CA95EAF7F6CF0E942014882319F00E94DA
:1035C000721A08950E945614CB0108956091DA038F
:1035D000669570E04BE050E084E391E00E94373064
:1035E000892B19F481E0809334030E94DB1A9093B5
:1035F0002E0380932D0380913503846080933503DF
:1036000008959091DA0390FF31C0917081112FC01D
:1036100092609093DA038091350381608093350343
:10362000662351F06091DA037091DB038091DC0333
:103630009091DD030E9422166091DA03669570E096
:103640004BE050E084E391E00E943730892BB1F0E9
:103650000E947A0881E08093300320E04091DD03EE
:103660006091DC038091DB030E943516089583325C
:1036700010F09464CECF880F982BCBCF0E94E61A1F
:10368000E9CF8091DA038695815009F482E261E006
:103690000E94011B08958091DA0386958F5F833223
:1036A00008F081E061E00E94011B08959091DA0327
:1036B00090FF08C09695981728F0961718F40E9466
:1036C0004B1B089561E00E94011B0895A5E0B0E046
:1036D000ECE6FBE10C946A2F8C01FC018381948160
:1036E000892B31F08081918189238F3F09F0EFC5CB
:1036F0002596E1E10C94862F0E949515F82E682FEF
:1037000089819A810E94540B69817A818F2D0E9450
:1037100087157C01F8018281882309F4CBC5C70194
:1037200082519F45409708F066C58FEF93E00E9455
:10373000F932811128C0FEEEEF0E57EA852E99244A
:103740009394E11032C01C821B82442443944AE0CB
:10375000342E74018FEFE81AF80AC4010E94F9327E
:1037600089831A82882379F09FEF980F933058F558
:103770008A83498292E0890E911CC7010E94F93226
:103780008B83811121C080917902877009F4B0CFB9
:10379000F8018281882309F4ABCF8091F10382FF85
:1037A000A7CF82E00E94CB0CA3CF811424E0920625
:1037B00051F3C4010E94F932811101C0EA943FEF34
:1037C000831A930ABECF4701FE0131967F01F701AC
:1037D0002081222309F4BDCF213009F047C0918117
:1037E0008281913031F4F2E0EF0EF11C0E947014EE
:1037F00007C0923049F422E0E20EF11C0E940A1048
:103800003FEFE31AF30AE3CF933031F432E0E30EF3
:10381000F11C0E94DD0FF4CF943021F08FEFE81AF5
:10382000F80AEECF92E0E90EF11C30E020E0B7019B
:103830006F5F7F4FF70141818053990B8A3091056B
:1038400050F021503109E0F28FE99FE00197F1F744
:1038500000C00000F6CF329EF001339EF00D11241F
:103860009C012E0F3F1F842F7B01E1CFE22FF0E060
:10387000E555FE4F5490822F86958695869590E06B
:10388000FC01E556FE4F64902770712C022E02C099
:10389000759467940A94E2F7E1E06E227724FC01C4
:1038A000E557FE4FA490B12C022E02C0B594A79408
:1038B0000A94E2F7F1E0AF22BB24FC01E558FE4F89
:1038C000C490D12C02C0D594C7942A95E2F721E088
:1038D000C222DD246114710419F081EE0E940A10E5
:1038E000A114B10419F086EE0E940A10852D0E94E1
:1038F0007014A114B10419F086EE0E94DD0F61145A
:10390000710419F081EE0E94DD0FC114D10409F495
:1039100077CF8CE26BCF81E00E94E70C0E94B20C63
:1039200032CF81E00E94BE0CF9CF82E0F5CFC70113
:103930007BC425EFE2162CE5F20609F46EC008F40C
:1039400068C027E245EE66EE86EFE8168CE5F806DD
:1039500009F4ACC4F8018281882309F4C9C4109227
:103960002604F3E0EF16FDE5FF0608F05DC02AEF40
:10397000E2162CE5F20630F4C70182509C454497CC
:1039800008F05FC00E9414169093F1038093F00337
:10399000E2E1EE16ECE5FE0609F474C108F0B2C0EF
:1039A00029E0E2162CE5F20609F44AC108F075C0D8
:1039B00085E0E8168CE5F80609F432C108F05FC02E
:1039C000E3E0EE16ECE5FE0609F422C108F024C19E
:1039D0008091F003816022E0E2162CE5F20609F402
:1039E0008EC06091F003F090F10384E090E00E94BB
:1039F0000D336F2D82E290E00E940D330E94F80C8F
:103A0000C2CE27E245EE65EE51C426E241EE60EEFD
:103A10004DC427E245EE64EE49C426E241EE62EE73
:103A200045C428E241E0EFCF35EAE3163DE5F30671
:103A300009F4A8CFF0F491E6E9169DE5F90609F43A
:103A4000A1CF86E1E8168CE5F80609F060C4809104
:103A50009B028A7A91E009F490E090932E0269E249
:103A6000811165E38EE092E00E9413080E944B0CE6
:103A70008ACEC7018D5A9D45039718F783CF809151
:103A8000F003806237E0E3163CE5F306C1F108F489
:103A9000D3C08091F003806432C09DE0E9169CE5BC
:103AA000F90609F4D7C0A0F48091F0038E7FFBE003
:103AB000EF16FCE5FF0619F18091F0038C602CE015
:103AC000E2162CE5F206D8F08091F0038D7F17C046
:103AD0003FE0E3163CE5F30609F4CCC008F4BEC0B1
:103AE00090E1E9169CE5F90609F4C8C08091F0035D
:103AF0008F7BE1E1EE16ECE5FE0609F072CF8093D4
:103B0000F0036FCFFFEFEF16FCE5FF0609F4C4C02A
:103B1000D8F53AEFE3163CE5F30609F485C0D0F496
:103B200094E1E9169CE5F90609F4C4C008F4B0C0B4
:103B3000F5E1EF16FCE5FF0609F053CF8091F003A5
:103B400082FB992790F921E0922790FB82F990FB64
:103B500083F9D5CF2CEFE2162CE5F20609F482C0EA
:103B600008F466C08DEFE8168CE5F80609F47EC00F
:103B70008091F10383609EEFE9169CE5F90609F058
:103B800030CF8093F1032DCFE1E6EE16EDE5FE0692
:103B900009F49BC0A0F421E0E2162DE5F20609F439
:103BA00092C008F47DC060E082E0E8168DE5F8067A
:103BB00009F017CF8EE090E00E940D3312CF9DEAFE
:103BC000E9169DE5F90601F168F49091F003892F5B
:103BD0008E7F90FF8160F5EAEF16FDE5FF0609F4A0
:103BE0008ECFFFCE2EEAE2162DE5F20679F13FEAFE
:103BF000E3163DE5F30609F0F4CE9091F103892F29
:103C0000877F93FF8860BDCF8091F1038860B9CF33
:103C10008091F003826073CF8091F00384606FCF56
:103C20008091F00388606BCF8091F1038160A9CF10
:103C30008091F1038260A5CF8091F00380615FCF16
:103C40000E94F80C8091F003806859CF8091F103B5
:103C5000877F97CF8091F0038B7F51CF8091F003C6
:103C6000877F4DCF8091F1038E7F8BCF8091F103C1
:103C70008D7F87CF8091F0038F7E41CF8091F003BD
:103C80008F7D3DCF0E94F80C8091F0038F7737CF66
:103C90008091F003837F33CF8091F1038C7F71CFCC
:103CA0008091F103982F909591708E7F892B90FBD6
:103CB00081F967CF0E94F80C9091F003892F97FB50
:103CC00087F980581CCF61E075CF9091F003892F60
:103CD0008F7E94FF806113CF81608093DA0361E06F
:103CE00086950E94011B4FCD41E45BE16BE47BE1D3
:103CF0000E94740848CD4BE45BE161E47BE1F8CFBE
:103D000044E057E16AEF76E1F3CF40EE56E16DEE25
:103D100076E1EECF46EC56E163ED76E1E9CF43ED97
:103D200056E166EC76E1E4CF40E257E16EE077E100
:103D3000DFCF61E081E0D5CF65E082E00E94561BD5
:103D400022CD68E086E0FACF64E18FE0F7CF67E14B
:103D500085E1F4CF62E289E1F1CF0E94F80C2FEF08
:103D600034E38CE0215030408040E1F700C0000097
:103D70000E94CC078091F10382FB882780F991E0B3
:103D800089270E943C15F8018281E080F180882318
:103D900009F445C0C7010E949515D82E682FC701A8
:103DA0000E94540BB7018D2D0E9487150E9489092E
:103DB0007C01882EF801D280B580B2943FE0B32216
:103DC000809179028770C1F0AD2CDD20B1F08F2D8C
:103DD000807F803421F080E28E0D883068F0809101
:103DE000F10382FF09C082E00E94CB0C809179022E
:103DF0008770AA24A3948111A12C9F2C92942FE068
:103E00009222FBE0F91508F479C0E92DF0E0E35BBC
:103E1000FC4C0C94F02F81E0B4CF80E0B2CFC7010E
:103E20000E94200BD82EBECF2F2D2F70C22E8F2D8B
:103E3000807F19F0C29490EFC922DD20B9F0CC2028
:103E400069F080E28E0D883010F0811009C08091F9
:103E50009B02C82AC0929B020E944B0C8E2D4CC024
:103E600080919A02C82AC0929A02F6CF8E2D0E94A3
:103E7000DD0FCC2009F442C080E28E0D883010F0B6
